:100000004D298030A100FE30AF200130AF20753087
:10001000AA0030300229A101A117B200B208031DC5
:100020001328030114280130B2020310A20CA20C01
:10003000A20CC0302205403EB207FE30AF2032088D
:10004000AF28A101A117B200FE30AF203208AF28BF
:10005000A401AD00AE01A01124080319A0150530BC
:10006000A3002730AC00103041200330AC00E83052
:100070004120AC0164304120AC010A3041202D0800
:100080004828AB002E08AA002D08A900162129082F
:10009000A900A3030319A01124080319522823025D
:1000A000031859282908031DA011A0195928303E0A
:1000B000AF280800A3002408031948292308AF200B
:1000C000A4035B28B0000611861183160611861161
:1000D0000F30860583123008A0188C283E30AA0005
:1000E000803002213330AF00A0201330AA008830C6
:1000F0000221A02064300121A0206430012122309F
:10010000AF00A02028308B200C308B2006308B20B5
:10011000A01430088C282014AF00201C9A288611C7
:10012000033C031C9F289F200530AA00DC300221DD
:10013000031408002014FE3C0319AD288615201C6A
:10014000201006150F3086052F08F0398604061199
:10015000AF0E2018A0283230012130084829A11BF9
:100160006228AC00220884002509841780058413C6
:10017000AC080319D928F030AE002B088038AD0048
:10018000F030AE030319AE000319AC030319D928EC
:10019000C928E420030126182508AB1F2508AB0851
:1001A00003190301AD0FD6288006BD28D72800000B
:1001B000C028250884178004482983178001840AF1
:1001C000FF3E031DDE284829270826040319A60A36
:1001D0008030261AA7062619A706A618A706270DF7
:1001E000A60DA70D26084829AC01AB00FF30AB07D0
:1001F000031CAC07031C48290330AA00DF3002218E
:10020000F628AA01E83EA900AA09FC30031C0B2924
:10021000A90703180829A9070000AA0F0829291807
:100220001129A91C1529000015290800AE01AD01EE
:100230001030AF002A0DAD0DAE0D2B08AD022C080D
:10024000031C2C0FAE0203182C292B08AD072C0819
:1002500003182C0FAE070310A90DAA0DAF0B1A2916
:10026000290848291030B300AA01A901B00CAF0C2D
:10027000031C40292B08A9072C0803182C0FAA07D8
:10028000AA0CA90CAE0CAD0CB30B36292D084829CD
:1002900083138312031300000800A00107309F009E
:1002A000B13083168500FF30860081132030840032
:1002B00060308312DE20A03084005030DE202030F9
:1002C00084003030DD20C830F4200120533062201B
:1002D00065306220613062207230622063306220BB
:1002E00068306220203062207330622069306220E2
:1002F000673062206E306220613062206C30622094
:1003000039140C2AC5013E03A800C9014908280276
:10031000031C9B29BE21B91C99294508A90049083D
:10032000A200A901A20A0314A90DA20B942929086D
:10033000C504C90F8629B5014508B400B50CB40C35
:10034000B50CB40CB50CB40CB50CB40C0F30B50531
:100350003508B0003408AF00AC010A30AB003221E0
:10036000B4002E08B500B7014508B6000F30B60539
:100370000030B70534083607C5000800BD01BC01D0
:100380000618D3290130F420BC0A0319BD0A0B302A
:100390003D02031CD229031DD129B9303C02031CA4
:1003A000D229B12CC0299B30F4200618B914061CA0
:1003B000B910391CFE29B5014608B400B7013C301C
:1003C000B6000430A9000310B70CB60CA90BE32942
:1003D000B60A0319B70A3508AA003408A900370875
:1003E000AC003608AB001621BF008030A1000230FF
:1003F000A2003F080D20FF306220062A8030A100B5
:100400008E3021200230A40046082920C60A051596
:100410001E30F42005110800C101C6013911391937
:10042000AB2ABD01BC01061C262ABC0A0319BD0A61
:100430000130F420AF303D02031C252A031D242A7D
:10044000C9303C02031C252AB12C132ABD01BC0172
:1004500006185A2ABC0A0319BD0A0A30F4203918B2
:100460004E2A3C08613A3D04031D402A8030A10019
:100470008E302120353062203930622005154D2A1A
:100480003C08643A3D04031D472A05114D2A3C08E7
:10049000FA3A3D04031D4D2AB12C592A11303D0270
:1004A000031C592A031D582A95303C02031C592A63
:1004B000B12C282A3D304102031C5F2AB12CC10A0D
:1004C0003D08031D672A65303C02031C682A391564
:1004D000391CAA2AB5014108B400B7013D30B60065
:1004E0000430A9000310B70CB60CA90B722AB60A87
:1004F0000319B70A3508AA003408A9003708AC0068
:100500003608AB001621BF008030A10080302120CA
:10051000463062206F306220753062206E3062207B
:1005200064306220203062207330622069306220A3
:10053000673062206E306220613062206C30622051
:10054000203062208030A1000230A2003F080D2040
:10055000FF3062200F2A391CCF2A01204930622047
:100560006E3062206930622074306220693062200F
:10057000613062206C306220693062207A30622003
:10058000653062202E306220622062208030A1001F
:10059000C03021200E30A4005F305A20FD2A0930DF
:1005A000BF000130A2003F080B20A1010A30420227
:1005B0000318DC2A203062208030A1004208282065
:1005C0003A3062200230A400430829203A306220E9
:1005D0003030622062204308031DEF2A812C1E3038
:1005E000430203190130031D0301B80003018618FB
:1005F000013038050319FD2A812C391D7F2CC901D2
:100600000F3049020318072BBE21C90F002BBE2152
:10061000BE21BE21B91C0E2B85150F2B8511123062
:10062000C900143049020318182BBE21C90F112B21
:10063000BE210730BE0082214508C300BE2106301E
:10064000BE0082214508C200BE210630BE008221C4
:100650004508C0000330BE0082214508C7000530B0
:10066000BE0082214508C4000830BE008221450832
:10067000C800BE21391C3E2B391001208030A1005A
:10068000803021200830A40020305A208030A10082
:10069000C03021201030A40020305A20803021208A
:1006A000A10101304702031D5C2B4D3062206F30E9
:1006B00062206E3062209D2B02304702031D672BA3
:1006C0005430622075306220653062209D2B0330EB
:1006D0004702031D722B5730622065306220643060
:1006E00062209D2B04304702031D7D2B5430622075
:1006F00068306220753062209D2B05304702031D53
:10070000882B4630622072306220793062209D2B27
:1007100006304702031D932B533062206130622064
:10072000743062209D2B07304702031D9D2B5330F0
:100730006220753062206E3062208030A100C030AF
:100740002120400828202030622001304402031D6F
:10075000B82B4A306220613062206E3062207530E2
:100760006220613062207230622079306220742C05
:1007700002304402031DCD2B4630622065306220DA
:1007800062306220723062207530622061306220F7
:100790007230622079306220742C03304402031DD1
:1007A000DC2B4D3062206130622072306220633079
:1007B000622068306220742C04304402031DEB2B4D
:1007C00041306220703062207230622069306220D5
:1007D0006C306220742C05304402031DF62B4D3022
:1007E00062206130622079306220742C063044022D
:1007F000031D032C4A306220753062206E30622067
:1008000065306220742C07304402031D102C4A30DE
:100810006220753062206C30622079306220742C46
:1008200008304402031D212C4130622075306220C3
:10083000673062207530622073306220743062202D
:10084000742C09304402031D382C5330622065306B
:1008500062207030622074306220653062206D301A
:100860006220623062206530622072306220742C17
:100870000A304402031D4B2C4F306220633062204B
:10088000743062206F3062206230622065306220F6
:1008900072306220742C0B304402031D602C4E30E9
:1008A00062206F30622076306220653062206D30C9
:1008B0006220623062206530622072306220742CC7
:1008C0000C304402031D742C4430622065306220D9
:1008D00063306220653062206D30622062306220B9
:1008E0006530622072306220203062202730622022
:1008F0008030A1000230A40048082920802CB12CAF
:100900000C2A0F30BF008514C6010F3046020318B1
:10091000B02C0530A2004030A5007F30AB00143071
:10092000B1208030A1000130A2003F080D2002302C
:10093000A4004608292005150530A2004030A50076
:100940007F30AB000230B120851005110530A200C8
:100950004030A5007F30AB003A30B120C60F852C67
:10096000072B01204E3062206F3062202030622041
:100970007330622069306220673062206E306220FE
:10098000613062206C306220203084006030DE20D4
:10099000A03084005030DE20203084003030DD2054
:1009A0000618B915061CB91103010618013EB9193C
:1009B000013C031DE12CBA0A0319BB0A0130F420E3
:1009C000D42C0301B9190130013A0319B911031DDF
:1009D000B91503010618013EB919013C031DF62C97
:1009E000BA0A0319BB0A0130F420E92C03303B0298
:0E09F000DE3003193A020318C42C39140C2A05
:02400E00503F21
:00000001FF
